S014000045696E646F706472616368742E737265633B
S113000045C0000049C100005EC000005CC00000A3
S11300105AC0000058C0000056C0000054C0000080
S113002052C0000092C100004EC000004CC000004D
S11300304AC0000048C0000046C0000044C00000A0
S113004042C0000040C000003EC000003CC00000B0
S11300503AC0000038C0000036C0000034C00000C0
S113006032C0000030C000002EC000002CC00000D0
S11300702AC0000028C0000026C0000024C00000E0
S113008022C0000020C000001EC0000011241FBEBA
S1130090CFEFD0E1DEBFCDBF11E0A0E0B1E0EEEDE7
S11300A0FAE000E00BBF02C007900D92A631B10741
S11300B0D9F721E0A6E1B1E001C01D92A232B20756
S11300C0E1F711D10AC59CCF9BB321E030E002C017
S11300D0220F331F8A95E2F7292B2BBB08959BB37C
S11300E021E030E002C0220F331F8A95E2F7209509
S11300F029232BBB089586E090E0E6DF83EC99E0AA
S11301000197F1F700C0000086E090E0E8DF87E89F
S113011093E10197F1F700C000000895CF93C82F31
S113012085BB84E090E0D0DFE6DFC295C07FC5BB2D
S113013084E090E0C9DFDFDFCF910895CF93C82F2B
S113014085BB84E090E0CBDFD6DFC295C07FC5BB22
S113015084E090E0C4DFCFDFCF91089581E0EEDF4B
S113016087E893E10197F1F700C0000080E8E6CF4B
S11301700895CF938FEF84BB85BB8ABB15BA1BBA96
S1130180C0E2C5BBB8DFC5BBB6DF80E885BBB3DF63
S113019015BAB1DF80EF85BBAEDF15BAACDF80E600
S11301A085BBA9DF82E0CADFA6DFCF910895CF9394
S11301B0DF93EC0102C0B2DF219688818111FBCF6D
S11301C0DF91CF910895AF92BF92CF92DF92EF92D9
S11301D0FF920F931F93CF93DF93CDB7DEB7D82E43
S11301E0C92EADB6BEB69F938F930F2EF2E1EF2EBC
S11301F0F1E0FF2EF02DFF92EF921F921F921F92BB
S11302001F9282D101962DB73EB7285F3F4F0FB69C
S1130210F8943EBF0FBE2DBF281B390B0FB6F894C0
S11302203EBF0FBE2DBF0DB71EB70F5F1F4FCF923E
S1130230DF92FF92EF929F938F931F930F9364D15A
S1130240802F912FB4DF8DB79EB708960FB6F89420
S11302509EBF0FBE8DBF0FB6F894BEBE0FBEADBE1F
S1130260DF91CF911F910F91FF90EF90DF90CF908E
S1130270BF90AF90089520910001222351F001977F
S1130280439738F4D1D01092000161E080E092E00D
S1130290BEC0089504C108951F920F920FB60F9225
S11302A011240BB60F922F933F934F935F936F9349
S11302B07F938F939F93AF93BF93EF93FF93FCD060
S11302C0FF91EF91BF91AF919F918F917F916F912A
S11302D05F914F913F912F910F900BBE0F900FBEE6
S11302E00F901F901895CCD044DFA0D08AE491E001
S11302F027D08BE391E0FED087EA91E60197F1F7EE
S113030000C000002BDF60E088E592E080D026DFAB
S1130310F6D059DF84E690E0A4D0F9CF90911D0186
S1130320911107C0E82FF0E0EF5FFE4F808183B9A1
S11303300895E82FF0E0E75FFE4F808183B90895C8
S113034090931F0180931E0108951F920F920FB680
S11303500F9211240BB60F922F933F934F935F93F9
S11303606F937F938F939F93AF93BF93EF93FF9379
S113037014BC80911601D2DF80911601873020F4DD
S11303808F5F8093160130C010921601809117017F
S113039090911801009799F480911D01811104C076
S11303A081E080931D0102C010921D01809119010A
S11303B090911A01909318018093170115C09C0124
S11303C02F713327232B39F4E0911E01F0911F0183
S11303D0309709F0099580911701909118010197C0
S11303E09093180180931701FF91EF91BF91AF9102
S11303F09F918F917F916F915F914F913F912F9139
S11304000F900BBE0F900FBE0F901F9018959093F6
S113041018018093170190931A0180931901609336
S11304201D018CE085BD089515BC08958FEF82B938
S11304308093640081E08093650013B886E983BDEE
S113044080E887BF7894089520E030E006C043E058
S11304504A95F1F700002F5F3F4F28173907B8F38B
S1130460089520E030E008C0E3ECF9E03197F1F7BB
S113047000C000002F5F3F4F28173907A8F30895E5
S11304808FEF8093640011BA83E080936A0089B788
S1130490816089BF1FBC8CE08EBD78940895CF9392
S11304A0DF93C5E6D0E018828AE090E0CDDF81E0FA
S11304B08883DF91CF91089580911101813041F4B7
S11304C082E080936A001DBC1CBC10921101089547
S11304D083E080936A008CB59DB590931C01809352
S11304E01B01E0912001F0912101099581E08093A5
S11304F01101089590932101809320010895809122
S11305001B0190911C0108950F931F93CF93DF93C8
S1130510CDB7DEB72E970FB6F894DEBF0FBECDBFB2
S11305200D891E898F89988D26E02C831A8309836F
S113053097FF02C080E090E801979E838D83AE010F
S1130540455E5F4F698D7A8DCE01019619D04D813C
S11305505E8157FD0AC02F813885421753070CF47A
S11305609A01F801E20FF31F10822E960FB6F89449
S1130570DEBF0FBECDBFDF91CF911F910F910895C4
S11305802F923F924F925F926F927F928F929F929F
S1130590AF92BF92CF92DF92EF92FF920F931F938D
S11305A0CF93DF93CDB7DEB72B970FB6F894DEBFAA
S11305B00FBECDBF6C017B018A01FC01178216823C
S11305C0838181FFBFC1CE0101963C01F601938175
S11305D0F70193FD859193FF81917F01882309F4AD
S11305E0ADC1853239F493FD859193FF81917F01EB
S11305F0853221F4B60190E0D6D1E8CF912C212C9C
S1130600312CFFE1F315D8F08B3279F038F48032D5
S113061079F08332A1F4232D20611DC08D3261F065
S1130620803369F4232D216016C0832D8260382E17
S1130630E32DE4603E2E2AC0F32DF8601DC037FC84
S11306402DC020ED280F2A3040F08E32B9F436FC4C
S113065075C1232D2064322E19C036FE06C08AE0EF
S1130660989E200D1124922E11C0EAE02E9E200D9A
S11306701124222EF32DF0623F2E08C08C3621F473
S1130680832D8068382E02C0883641F4F70193FD2B
S1130690859193FF81917F018111B3CF982F9F7D25
S11306A09554933028F40C5F1F4F9FE399830DC03A
S11306B0833631F0833771F0833509F055C020C09B
S11306C0F801808189830E5F1F4F88248394912CC5
S11306D0530112C02801F2E04F0E511CF801A08012
S11306E0B18036FE03C0692D70E002C06FEF7FEF6A
S11306F0C5014ED14C018201F32DFF773F2E15C069
S1130700280122E0420E511CF801A080B18036FE7F
S113071003C0692D70E002C06FEF7FEFC5012DD1DA
S11307204C01F32DF0683F2E820133FC19C0822D59
S113073090E088169906A0F4B60180E290E033D1E7
S11307402A94F5CFF50137FC859137FE81915F013D
S1130750B60190E028D121102A9421E0821A910850
S11307608114910479F7E1C0843611F0893639F5A2
S1130770F80137FE07C060817181828193810C5F2B
S11307801F4F08C060817181072E000C880B990BE4
S11307900E5F1F4FF32DFF763F2E97FF09C09095F4
S11307A08095709561957F4F8F4F9F4FF0683F2ED6
S11307B02AE030E0A30133D1882E861844C085375F
S11307C031F4232D2F7EB22E2AE030E025C0932D64
S11307D0997FB92E8F36C1F018F4883579F0AEC000
S11307E0803719F0883721F0A9C0E92FE061BE2EC7
S11307F0B4FE0DC0FB2DF460BF2E09C034FE0AC048
S1130800292F2660B22E06C028E030E005C020E182
S113081030E002C020E132E0F801B7FE07C0608199
S11308207181828193810C5F1F4F06C06081718149
S113083080E090E00E5F1F4FA301F1D0882E861850
S1130840FB2DFF773F2E36FE0DC0232D2E7FA22ECB
S1130850891458F434FE0BC032FC09C0832D8E7EFB
S1130860A82E05C0B82CA32C03C0B82C01C0B92CE9
S1130870A4FE0FC0FE01E80DF11D8081803321F438
S11308809A2D997EA92E09C0A2FE06C0B394B394F2
S113089004C08A2D867809F0B394A3FC10C0A0FE8E
S11308A006C0B21480F4280C922C9B180DC0B2140C
S11308B058F4B60180E290E076D0B394F8CFB21445
S11308C018F42B1802C0982C212CA4FE0FC0B601DA
S11308D080E390E068D0A2FE16C0A1FC03C088E7C4
S11308E090E002C088E590E0B6010CC08A2D8678BD
S11308F051F0A1FE02C08BE201C080E2A7FC8DE2B0
S1130900B60190E050D0891430F4B60180E390E051
S11309104AD09A94F8CF8A94F301E80DF11D8081AE
S1130920B60190E040D08110F6CF222009F44ECEDB
S1130930B60180E290E037D02A94F7CFF6018681A1
S1130940978102C08FEF9FEF2B960FB6F894DEBF0E
S11309500FBECDBFDF91CF911F910F91FF90EF900C
S1130960DF90CF90BF90AF909F908F907F906F90CB
S11309705F904F903F902F900895FC010590615037
S113098070400110D8F7809590958E0F9F1F0895A1
S1130990FC016150704001900110D8F7809590954A
S11309A08E0F9F1F08950F931F93CF93DF93FB0127
S11309B0238121FD03C08FEF9FEF2CC022FF16C0BF
S11309C046815781248135814217530744F4A0811D
S11309D0B1819D012F5F3F4F318320838C9326810A
S11309E037812F5F3F4F3783268314C08B01EC017F
S11309F0FB010084F185E02D0995892BE1F6D801EE
S1130A0016968D919C911797019617969C938E93A9
S1130A101697CE01DF91CF911F910F910895FA019E
S1130A20AA27283051F1203181F1E8946F936E7F29
S1130A306E5F7F4F8F4F9F4FAF4FB1E03ED0B4E01A
S1130A403CD0670F781F891F9A1FA11D680F791F5B
S1130A508A1F911DA11D6A0F711D811D911DA11D6C
S1130A6020D009F468943F912AE0269F112430197C
S1130A70305D3193DEF6CF010895462F4770405D17
S1130A804193B3E00FD0C9F7F6CF462F4F70405DC6
S1130A904A3318F0495D31FD4052419302D0A9F721
S1130AA0EACFB4E0A6959795879577956795BA951B
S1130AB0C9F700976105710508959B01AC010A2EE1
S1130AC006945795479537952795BA95C9F7620FB8
S1110AD0731F841F951FA01D0895F894FFCF77
S1130ADE01080C0406020301090901030206040CB1
S1090AEE0801256400006C
S9030000FC
